:1000000008308A00202E0000FF00030E8301A100AB
:100010000A08A0008A010408A2007708A300780853
:10002000A4007908A5007A08A6007B08A70083131E
:1000300083128B1E1D280B193028220884002308E8
:10004000F7002408F8002508F9002608FA00270818
:10005000FB0020088A00210E8300FF0E7F0E09009E
:100060008A110A12C9280A108A100A118207443418
:1000700069346D344C3475346E344D3461347234BB
:100080004D34653472344A346534753456346534CD
:100090006E34533461346D3400340A108A100A11FE
:1000A000820700341E34253429341E3400340034D1
:1000B00011343F34013400341134233425341934DD
:1000C00000341E34253429341E340A108A100A11D3
:1000D00082074A344F34553420344834453455343B
:1000E000523445342034543445344D345034203463
:1000F0005034523445345334533400340A108A1087
:100100000A1182072B3433343534633400340A1037
:100110008A100A1182072B343234303463340034AD
:100120000A108A100A1182072034303463342034D4
:1001300000340A108A100A1182072D343134353404
:10014000633400340A108A100A1182072B343134C8
:100150003534633400340A108A100A1182072D34B2
:1001600032343034633400340A108A100A118207A2
:100170002D3433343534633400340A108A100A11B4
:10018000820720342D3430342E3425347534203415
:100190000034AD0BCF281030AD002814AE0A2E0865
:1001A0003B3C0318D928AE01AF0A2F081E3C0319A7
:1001B000A8142F083B3C0318E028AF01B00A28150B
:1001C0003008183C031DE628B001B10A3108063C8E
:1001D0000318EB28B1010B118A110A121D28A9017D
:1001E0002908113C031CFB284A3029078400FF30F2
:1001F0008000A90AF02883161F109F141F159F1551
:100200001F1383121F179F1783169F1783121F1424
:10021000850186018701FF30831685000030860046
:100220000F30870083122810A8102811A81581010B
:100230000730F700F71D2429073081018130840041
:100240000008C0390F388000640081308400000845
:10025000C039770480008B16C0308B048A150A12CF
:10026000372E5F3084000008031943290130F8005D
:10027000F701F70B3929F80B38295B30F700F70B3A
:100280003F29800B36290034FF3083168600831205
:10029000871787120713000000000608B40007172D
:1002A0000000000087160030831686008312003499
:1002B0004421600886008713071207130000071700
:1002C00007164421610886008713071207130000F0
:1002D0000717071600344421710886008717071294
:1002E00007130000071707160034071687160717AD
:1002F000871705166430DF003121E101E001582144
:100300004030F1006B21E1011430E0005821413010
:10031000F1006B210430E100E00158214230F1008E
:100320006B21E1011430E00058214330F1006B21D2
:100330008030F1006B219C30F1006B218A150A128C
:100340003A2E442160088600871307120713000025
:1003500007170716C030F1006B210034E101E001FE
:1003600058212430F1006B21B801B70138081F3C37
:10037000031CC629031DC0293708FE3C031CC629DF
:10038000E001A121B70A0319B80AB629E101E00189
:1003900058212430F1006B218A150A12422E442183
:1003A000203070028600871307120713000007171A
:1003B0000716C030F1006B210034E101E001582143
:1003C0002430F1006B21DE015E086520DE0AF700B3
:1003D000F000CF2114305E02031DE4290430DF0059
:1003E00031210530E1005430E00058212430F10083
:1003F0006B212830A900A9080319032AFF30E00067
:10040000A121A903FB298A150A12452EF701F8013B
:100410005E0803105F18F707F70CF80CDF18F707F2
:10042000F70CF80C5F19F707F70CF80CDF19F70752
:10043000F70CF80C5F1AF707F70CF80CDF1AF70740
:10044000F70CF80C5F1BF707F70CF80CDF1BF7072E
:10045000F70CF80C00346208F80161020318332A23
:100460006108F7003F2AF7010830E300E10DF70DBE
:10047000620877020318F700F80DE30B362A003400
:100480006013E0125F08E1006430E2002B2277087D
:10049000DF007808031D6A2AE01A6A2AE019782A20
:1004A000601B582A6018582A6019582AE01B782ABD
:1004B000601C642AE01B782A601B642A6018782A72
:1004C0006019642AE01B782A2030601E3030F0006A
:1004D000CF21782AE016E01F742A78088000F800FF
:1004E0002D30F000CF21E01330307807F000CF211D
:1004F000601B832A5F08E1000A30E2002B227708A4
:10050000DF006017492AE01F882A2D30F000CF2134
:1005100030305F07F000CF2100340B138B138B1B9F
:100520008E2A0708FF3A0F39013A0319A12A033A24
:100530000319A22A063A0319A82A0C3A0319AE2A6B
:10054000B42AB52AB10A3108063C031CB101B52A08
:10055000B00A3008173C031CB001B52AAF0A2F08B7
:100560003B3C031CAF01B52AB52AE1011430E00081
:1005700058212430F1006B213108DE000330DF0008
:1005800006227808A9000330AA00AA080319D02A75
:1005900029083320DE00F000CF21A90AAA03C52ACA
:1005A0002030F000CF213008DF000130E000402291
:1005B0003A30F000CF212F08DF000130E000402268
:1005C0000230DE00FA30DF003121DE0BE22A00309B
:1005D000851A0130003A0319912AAE01C0308B040C
:1005E0008A150A12592EDE080319FC2A85143D309B
:1005F00083168500FF2A83123F30831685008312FD
:10060000003485103D3083168500F430F700F70B79
:10061000072B3F308500D130F700F70B0D2B000082
:10062000831200340830DF000310DE0C031C292B7A
:1006300085103D30831685000330F700F70B1E2B25
:100640003F3085001430F700F70B242B0000332BCC
:10065000831285103D30831685001830F700F70BA4
:100660002F2B3F3085008312DF03DF08031D142B7F
:1006700000345E085F068039E100DE1F412BDE0991
:10068000DE0ADF1F452BDF09DF0A5F08F8015E0283
:1006900003184D2B5E08F700592BF7010830E000D6
:1006A000DE0DF70D5F0877020318F700F80DE00B79
:1006B000502BE11F5D2BF809F80A000000348E3042
:1006C000F7005F08F8005E08F900FA01F808031D5A
:1006D000732B7908F800F9010830F702F808031DB8
:1006E000732BF7017B2B0310F81B7A2BF90DF80DF8
:1006F000F703732BF81300008A110A12902E5E087C
:100700000319442CEA0062080319442CEA02031C72
:100710008E2B7F30EA070318442C942B8130EA0299
:10072000031C442C0319442C6A08F700F801F90152
:10073000FA01E9015F08E800E8176008E7006108CE
:10074000E6001930EA006508E6020318B72B01300D
:10075000E7020318B72BE8020318B72BE9020318C6
:10076000B72BE90AE80AE70A6508E607E92B6408F7
:10077000E7020318D22B0130E8020318D22BE9025A
:100780000318D22BE90AE80A6408E7076508E607B8
:10079000031CE92BE70A031DE92BE80A031DE92BDB
:1007A000E90AE92B63088038E8020318E82B0130D6
:1007B000E9020318E82BE90A63088038E8076408AF
:1007C000E707031CC62BE80A031DC62BE90AC62B44
:1007D0007A14EA0BEC2BF72B0310E60DE70DE80D6E
:1007E000E90D0310FA0DF90DF80DEB0DA32B6B1CA1
:1007F000FF2B0310F80CF90CFA0CEB0C022CF7038E
:100800000319442CEB1B2B2C0310E60DE70DE80D10
:10081000E90D6508E6020318172C0130E7020318FA
:10082000172CE8020318172CE902031C3A2C640861
:10083000E7020318222C0130E8020318222CE902F7
:10084000031C3A2C63088038E80203182B2C013073
:10085000E902031C3A2CFA0A031D3A2CF90A031D7B
:100860003A2CF80A031D3A2CF70A0319442CF80C09
:10087000F90CFA0C5F08EA006308EA06EA1F422C4A
:10088000F817482CF813482CF701F801F901FA0180
:1008900000008A110A12A12E80308318E306E801B5
:1008A000E9015F08E7006308E7065E080319392DD0
:1008B000E600F70062080319422DE6020319DF2C57
:1008C000031C9E2C6308EC00EC176408EB00650821
:1008D000EA00E9010310EC0CEB0CEA0CE90CE60B66
:1008E000692CE71F762C6814562D68106610681660
:1008F000613084006B2D6812E71B882C661C932CDA
:10090000EC0CEB0CEA0CE90CF70A0319512D932CB3
:10091000EC1B962C0310E90DEA0DEB0DEC0DF70323
:100920000319512D882C6817FE2C68135F08E70007
:10093000DF1F9C2CEC174A2DEC134A2D6208E600B1
:10094000F7005E08E6025F08EC00EC176008EB00B9
:100950006108EA00E9010310EC0CEB0CEA0CE90C6D
:10096000E60BAA2CE71FB72CE814562DE8106610EA
:10097000E816653084006B2DE812E71BC92C661C55
:10098000D42CEC0CEB0CEA0CE90CF70A0319512DF2
:10099000D42CEC1BD72C0310E90DEA0DEB0DEC0D5C
:1009A000F7030319512DC92CE817FE2CE81363082F
:1009B000E700E31FDD2CEC174A2DEC134A2D6308EA
:1009C000EC00EC176408EB006508EA00E71FEC2C6C
:1009D000EC136815562D6811E9016610613084002A
:1009E0006B2DE71B142D5F08E700661CFE2CEC0C3A
:1009F000EB0CEA0CE90CF70A0319512DE91F0F2D36
:100A0000EA0A031D0F2DEB0A031D0F2DEC0A031D2F
:100A10000F2DEC0CEB0CEA0CF70A0319512D681B97
:100A2000952CE81BD62C332D8030EC06EC1F1C2DAA
:100A3000562D6308E700292D5F08E700EC08031D29
:100A4000292DEB08031D292DEA08031D292DF70187
:100A50004A2DEC1B332D0310E90DEA0DEB0DEC0DC7
:100A6000F70B292D512DE71F372DEC174A2DEC13CD
:100A70004A2D6208F7006308EC006408EB00650883
:100A8000EA004A2D5E08F7005F08EC006008EB0002
:100A90006108EA006C08F8006B08F9006A08FA00BF
:100AA000892DF701F801F901FA01892DE901EA0917
:100AB000EB09EC09E909E90A031D642DEA0A031DA3
:100AC000642DEB0A0319EC0A6818752CE818B62C8B
:100AD0006819EB2C192D0008EA07031C752DEB0A89
:100AE000031D752DEC0A0319661484030008EB0737
:100AF000031C7D2DEC0A0319661484030008801F73
:100B0000803AEC0703186614681A7B2CE81ABC2C90
:100B1000F12C00008A110A12B92E0030F8001F08CB
:100B2000C73978049F00DE01F32200000000012392
:100B3000CC30DE001223BE30DE001223DE01DF01E6
:100B40001030E000E0080319BF2D85103D308316FA
:100B500085003F308500000000000000000000001C
:100B600083128518B52D0310B62D0314DF0CDE0C8F
:100B70001B30F700F70BBA2D0000E003A22D5E0832
:100B8000F8005F08F9007808B9000123CC30DE00D6
:100B900012234430DE0012230130DE00F322390834
:100BA000DE000230DF0039237808BA003908DE00A1
:100BB0000230DF00392377080319E12D0530BB002F
:100BC000E22DBB013A08803A713C03182812BA1B87
:100BD000ED2D3A080E3C031C2816281E392EE10183
:100BE0003C30E00058212430F1006B21DE015E082A
:100BF0007E20DE0AF700F000CF2104305E02031DE4
:100C0000F72DE1017830E00058212430F1006B210C
:100C1000DE015E088720DE0AF700F000CF210430F5
:100C20005E02031D092EE101DC30E0005821243072
:100C3000F1006B21DE015E089020DE0AF700F00073
:100C4000CF2104305E02031D1B2E0130E10018305D
:100C5000E00058212430F1006B21DE015E0899206C
:100C6000DE0AF700F000CF2104305E02031D2E2EB5
:100C7000822EE1013C30E00058212430F1006B214C
:100C8000DE015E08A220DE0AF700F000CF2104306A
:100C90005E02031D412EE1017830E000582124302E
:100CA000F1006B21DE015E089020DE0AF700F00003
:100CB000CF2104305E02031D532EE101DC30E00041
:100CC00058212430F1006B21DE015E08AB20DE0AE2
:100CD000F700F000CF2104305E02031D652E0130C5
:100CE000E1001830E00058212430F1006B21DE01D2
:100CF0005E08B420DE0AF700F000CF2104305E0267
:100D0000031D782E1F151F19832E83161E088312AC
:100D1000B5001E08B6003608DF003508DE005F2B80
:100D20007A08E1007908E0007808DF007708DE0043
:100D30009A30E5009930E4004C30E3008530E20061
:100D40007F2B7A08BF007908BE007808BD007708BD
:100D5000BC0083103F08E1003E08E0003D08DF00D2
:100D60003C08DE00E501E4013E30E3008530E200AE
:100D70004C2C7A08BF007908BE007808BD007708BF
:100D8000BC008A150A125E2EDE1FCA2EDF17DE098E
:100D9000DE0AD12E5F1DD12E20305F1E3030F000D4
:100DA000CF215F13DF125E08E1006430E2002B22E6
:100DB0007708DE007808031DFB2EDF1AFB2EDF19F3
:100DC000092F5F1BE92E5F18E92E5F19E92EDF1B43
:100DD000092F5F1CF52EDF1B092F5F1BF52E5F18F7
:100DE000092F5F19F52EDF1B092F20305F1E3030D1
:100DF000F000CF21092FDF16DF1F052F78088000B4
:100E0000F8002D30F000CF21DF1330307807F000EC
:100E1000CF215F1B142F5E08E1000A30E2002B2275
:100E20007708DE005F17DA2EDF1F192F2D30F00054
:100E3000CF2130305E07F000CF2100345F08E6009C
:100E40006308E606E61F292F03110310DF1B0314B6
:100E50005C2F5F08E6006208E7005E08E7020319FE
:100E6000372FE61F5C2F0308013A83005C2F6308CD
:100E7000E7005F08E7020319432FE61F5C2F030812
:100E8000013A83005C2F6408E7006008E702031959
:100E90004F2FE61F5C2F0308013A83005C2F650883
:100EA000E7006108E70203195B2FE61F5C2F0308C8
:100EB000013A83005C2F03108A150A12792A053043
:100EC000C1009030C0000130A90029086C3C031C0F
:100ED000CA2F4108E1004008E00058212430F10009
:100EE0006B211430AA00AA080319982F01302A0296
:100EF0004A3EDF004421C130F1006B214421FF3024
:100F000083168600831287138712071300000000E0
:100F10000608E00007178716003083168600831244
:100F20006008F8005F08840078088000AA03732F27
:100F30000310CA0DCB0DCC0DCD0DCE0DCF0DD00DA8
:100F4000D10DD20DD30DD40DD50DD60DD70DD80D95
:100F5000D90DDA0DDB0DDC0DDD0D4108E100400897
:100F6000E00058212430F1006B211430AA00AA08B7
:100F70000319C42F01302A024A3E84000008DF0012
:100F8000E000A121AA03B72F1430C0070318C10A3B
:100F9000A90A652F00341030F700FA01E201DF0CD6
:100FA000DE0C031CD92F6008FA070318E20A610857
:100FB000E207E20CFA0CF90CF80CF70BCF2F003417
:101000006208EB006308EC00ED01DF1F09286B1795
:10101000EC03DF175E080319AC287F305E02031C67
:101020006828DE00EE010430EF000310E10DE00D52
:10103000DF0DED0DEF0B152804305E020318282894
:1010400003305E02031DA2280A306D02031CA22891
:101050000330DE02EE0A7D210310E10DE00DDF0D0D
:10106000ED0D66210230EF000310ED0CDF0CE00CFB
:10107000E10CEF0B34287D210430EF000310E20C6B
:10108000E30CE40CE50CEF0B3E2866217D2164089F
:10109000E5006308E4006208E300E20166217D21C7
:1010A0006308E5006208E400E201E3016621ED194E
:1010B0001C28DE08031D6128E10AE00ADF0AED0AA8
:1010C000A2280310E10DE00DDF0DED0DDE031C285D
:1010D000DE09DE0A7F30DE07EE010430EF00031088
:1010E000E10DE00DDF0DED0DEF0B6F280430DE0795
:1010F00005305E02031CAE287D210310E10DE00DDA
:10110000DF0DED0D0310E10DE00DDF0DED0D66219E
:101110000310E10DE00DDF0DED0DEE0A0330EF00E1
:101120000310ED0CDF0CE00CE10CEF0B902803300A
:10113000DE026D1E78280310ED0CDF0CE00CE10CD4
:10114000DE037828DE09DE0A0330DE076E0AEC02D1
:10115000031CEC010130AF280230AF280030E7005B
:10116000EB1BBE28EC1BBE28EC080319BE28203060
:10117000F0008A11CF218A15EC0BB7286B1FC52808
:101180002D30F0008A11CF218A15EB1FD328EC1BDC
:10119000D328EC080319D3283030F0008A11CF216E
:1011A0008A15EC0BC928EB136B13671CDE286E083D
:1011B000E7006E08E9006B0AE9070A29E71CE22844
:1011C0006B0AEE00EB08031964292E30F0008A1137
:1011D000CF218A156E08EA00EA036B086A02031C35
:1011E000F3286B08EA00EA080319FD283030F00004
:1011F0008A11CF218A15EA0BF6286E08EF006B0AD8
:10120000EF0203188629DE036B0AE9006E08E90283
:101210006908E7006D08E6005E0803191429E80074
:101220000310E60CE80B1029690803196429303013
:101230006607F0008A11CF218A156708031D282947
:10124000EB08031964292E30F0008A11CF218A158A
:10125000E703E903031964295E0803193429E80048
:101260000310E60DE80B30296608ED026D08E20078
:101270005F08E3006008E4006108E5000310E10D89
:10128000E00DDF0DED0D0310E10DE00DDF0DED0DB7
:101290006508E107031C5129E00F5129DF0F51298F
:1012A000ED0A6408E007031C5829DF0F5829ED0AEE
:1012B0006308DF070318ED0A6208ED070310E10D6C
:1012C000E00DDF0DED0D0A29000086296508E10714
:1012D000031C6F29E00F6F29DF0F6F29ED0A6408E7
:1012E000E007031C7629DF0F7629ED0A6308DF0784
:1012F0000318ED0A6208ED0700346D08E2005F088C
:10130000E3006008E4006108E500003400000034F8
:10131000E1011430E0008A1158218A152430F100CF
:101320008A116B218A153108DE000330DF008A1133
:1013300006228A157808A9000330AA00AA08031912
:10134000AD2929088A1133208A15DE00F0008A11A0
:10135000CF218A15A90AAA039E292030F0008A11FC
:10136000CF218A153008DF000130E0008A114022C9
:101370008A153A30F0008A11CF218A152F08DF0034
:101380000130E0008A1140228A15B91BE929390889
:10139000133C0318E9292030F0008A11CF218A1567
:1013A0003A08DE001830DF008A11C4268A152E3074
:1013B000F0008A11CF218A153B08DF001830E000C9
:1013C0008A1140228A152030F0008A11CF218A1517
:1013D000692AB91B0E2A2030F0008A11CF218A1504
:1013E0002030F0008A11CF218A153A08DE0018302B
:1013F000DF008A11C4268A152E30F0008A11CF2111
:101400008A153B08DF001830E0008A1140228A1557
:101410002030F0008A11CF218A15692A3908FF3C53
:10142000031D2E2ADE015E088A11BD208A15DE0A00
:10143000F700F0008A11CF218A1504305E02031DE7
:10144000132A3B08DF001830E0008A1140228A1579
:101450002030F0008A11CF218A15692A3908803A94
:101460006C3C031C4C2A3A08DE001830DF008A115D
:10147000C4268A152E30F0008A11CF218A153B0828
:10148000DF001830E0008A1140228A152030F00079
:101490008A11CF218A15692A2030F0008A11CF21C4
:1014A0008A153A08DE001830DF008A11C4268A1532
:1014B0002E30F0008A11CF218A153B08DF0018304A
:1014C000E0008A1140228A152030F0008A11CF21D5
:1014D0008A153F08E1003E08E0003D08DF003C08B7
:1014E000DE00E501E4014830E3008530E2008A11C6
:1014F0001E2F8A15031C912A2030F0008A11CF215B
:101500008A153F08E1003E08E0003D08DF003C0886
:10151000DE00E501E4010230E3000130E2000020DA
:10152000A02A3F08E1003E08E0003D08DF003C083B
:10153000DE00E501E4010330E3000130E2000020B9
:10154000A81DB22AE1011A30E0008A1158218A153B
:101550002430F1008A116B218A152A30F0008A119B
:10156000CF218A150030A8190130FF3EF800781805
:10157000BB2AA811BC2AA8158A150A12602E5E087B
:1015800003192F2BE600620803192F2BE607031817
:10159000D02A7F30E602031C2F2B03192F2BD42ACD
:1015A0008130E60703182F2B6608F700F801F901D0
:1015B000FA015F08EA00EA176008E9006108E8003C
:1015C0001830E600E701681CFD2A6508FA07031CCD
:1015D000EF2AF90A031DEF2AF80A0319E71764082E
:1015E000F907031CF62AF80A0319E7176308E00055
:1015F000E0176008F8070318E717E70DF80CF90C77
:10160000FA0CEA0CE90CE80C0310E60BE22A0130B4
:10161000F70703182F2BF81B142BEA0DFA0DF90D01
:10162000F80DF70303192F2BEA1F252BFA0A031DC8
:10163000252BF90A031D252BF80A031D252BF80C71
:10164000F90CFA0CF70A03192F2B5F08E70063085F
:10165000E706E71F2D2BF817332BF813332BF70171
:10166000F801F901FA0100008A150A12BF2B8E3029
:10167000F7005E08F7025F08F9006008F800F91744
:10168000F70803194E2B0310F908031D4A2BF8081D
:1016900003194E2BF90CF80CF70B432BDF1F552BBE
:1016A000F809F909F80A0319F90A00008A150A125B
:1016B000C82B281A652B46303907FA01F700F71BAB
:1016C000FA03C4007A08C5006E2B1E303907FA01F0
:1016D000F700F71BFA03C4007A08C500C51F722B78
:1016E000C501C401C51B7E2BC508031D7B2B440807
:1016F000643C03187E2BC5016430C4004408643C7C
:10170000C4000030F8004508031C450F892B7808F9
:101710008A2B7802C5004508DF004408DE00E1019D
:101720001430E0008A11CB278A157908C5007808A3
:10173000C400A330C4070318C50A0530C50745080F
:10174000E1004408E0008A1158218A152430F10094
:101750008A116B218A15F830F1008A116B218A15E4
:101760003F08E1003E08E0003D08DF003C08DE00E5
:10177000E501E4012030E3008230E200BF2A7A086C
:10178000E1007908E0007808DF007708DE00372BF9
:101790007908C5007808C400B630C4020330031CC1
:1017A0000430C502C51FD62BC501C401C51BE22BE1
:1017B000C508031DDF2B4408643C0318E22BC50158
:1017C0006430C4004408643CC4000030F80045089C
:1017D000031C450FED2B7808EE2B7802C500450859
:1017E000DF004408DE00E1011430E0008A11CB275D
:1017F0008A157908C5007808C400A330C407031807
:10180000C50A0530C5074508E1004408E0008A1113
:1018100058218A152430F1008A116B218A15F8307D
:10182000F1008A116B218A1514304407DE00450847
:10183000DF000318DF0A5F08E1005E08E0008A119C
:1018400058218A152430F1008A116B218A15F8304D
:10185000F1008A116B218A1500343008153C031CF5
:10186000352C3008023C031C852C32088A114D208F
:101870008A15F800B3000D30C500FF30C400C70161
:10188000C601C708031D842C4608053C031C842C94
:10189000DF011430DE004708E1004608E0008A114D
:1018A000CB278A157908FA0078084402DE0045083B
:1018B000DF007908031C790FDF025F08E1005E0892
:1018C000E0008A1158218A152430F1008A116B2119
:1018D0008A153308F7004608F8000319732C031023
:1018E000F70CF80B6F2C771C7B2CF830F1008A1169
:1018F0006B218A15802CF030F1008A116B218A153A
:10190000C60A0319C70A412CB20A3008093C031859
:10191000DD2C30080E3C031CDD2C32088A114D20D2
:101920008A15F800B3000D30C500FF30C400C701B0
:10193000C601C708031DDC2C4608053C031CDC2C33
:10194000DF011430DE004708E1004608E0008A119C
:10195000CB278A157908FA0078084402DE0045088A
:10196000DF007908031C790FDF025F08E1005E08E1
:10197000E0008A1158218A152430F1008A116B2168
:101980008A153308F7004608F8000319CB2C03101A
:10199000F70CF80BC72C771CD32CF830F1008A1108
:1019A0006B218A15D82CF030F1008A116B218A1531
:1019B000C60A0319C70A992CB20A00343008003A43
:1019C0000319EC2C063A03191D2D0A3A03194F2D61
:1019D0001E3A0319812DB32DB2010530C500A33085
:1019E000C400C701C6014708073C031C1C2D031D8A
:1019F000FD2C4608D03C031C1C2D46084407DE0085
:101A00004508DF000318DF0A4708DF075F08E10029
:101A10005E08E0008A1158218A152430F1008A11ED
:101A20006B218A15F830F1008A116B218A15283054
:101A3000C6070318C70AF32CB42D0630B2000530D0
:101A4000C500A330C400C701C6014708073C031CFA
:101A50004E2D031D2F2D4608D03C031C4E2D46084D
:101A60004407DE004508DF000318DF0A4708DF07E8
:101A70005F08E1005E08E0008A1158218A152430D1
:101A8000F1008A116B218A15F830F1008A116B215F
:101A90008A15C830C6070318C70A252DB42D0A3089
:101AA000B2000530C500A330C400C701C601470815
:101AB000073C031C802D031D612D4608D03C031CF0
:101AC000802D46084407DE004508DF000318DF0AC2
:101AD0004708DF075F08E1005E08E0008A1158212F
:101AE0008A152430F1008A116B218A15F830F10033
:101AF0008A116B218A156430C6070318C70A572D4F
:101B0000B42D1030B2000530C500A330C400C701A9
:101B1000C6014708073C031CB22D031D932D460840
:101B2000D03C031CB22D46084407DE004508DF0008
:101B30000318DF0A4708DF075F08E1005E08E000DE
:101B40008A1158218A152430F1008A116B218A15D7
:101B5000F830F1008A116B218A15C830C6070318C6
:101B6000C70A892DB42DB42D30080139003A031D60
:101B70001D2E0530C500A330C400C701C6014708AB
:101B8000023C031CEA2D031DC92D4608583C031CCA
:101B9000EA2D46084407DE004508DF000318DF0A87
:101BA0004708DF075F08E1005E08E0008A1158215E
:101BB0008A152430F1008A116B218A15F830F10062
:101BC0008A116B218A155830C6070318C70A0230DC
:101BD000C707BF2D7830C4070318C50A0530C507ED
:101BE000C701C6014708023C031C1D2E031DFC2D26
:101BF0004608583C031C1D2E46084407DE004508D5
:101C0000DF000318DF0A4708DF075F08E1005E080E
:101C1000E0008A1158218A152430F1008A116B21C5
:101C20008A15F830F1008A116B218A155830C607E1
:101C30000318C70A0230C707F22D8A150A12702E40
:101C400084011F30830583161F149F141F159F11D5
:101C500007309C001C0883120D1328160830AD00B5
:101C6000AE01AF01B001B101B2018A11EF288A15AE
:101C70008A1175298A15C830DF008A1131218A1529
:101C80008A11AE298A158A11DD298A150030851A34
:101C90000130003A031D5A2E1930DF008A1131211C
:101CA0008A150030851A0130003A031D5A2E8A1118
:101CB0008D2A8A15281C612E8A118D2D8A15882956
:101CC0002810A81C692E8A115F278A1559232D24F4
:101CD000A810281D722E8A115F278A155923DE2C21
:081CE0002D242811462E63009B
:02400E00713F00
:00000001FF
